:1000000044C068C067C025C324C323C322C362C0E1
:1000100061C060C05FC05EC05DC05CC0D0C25AC07D
:1000200059C058C057C056C000002E0025002800F7
:100030002B00040404040404040402020202020269
:10004000020203030303030303010101010301028D
:100050000408102040800102040810204080800124
:100060000204081020010204084000000000000003
:100070000000000304000000000000000000000079
:1000800000000000000005058C0511241FBECFEF05
:10009000D2E0DEBFCDBF22E0A2EEB1E001C01D92F2
:1000A000AC35B207E1F711E0A0E0B1E0E4EFF0E138
:1000B00002C005900D92A23EB107D9F710E0C4E44A
:1000C000D0E003C02197FE0118D6C334D107D1F781
:1000D0006CD304C895CF10924E0210924D0210922C
:1000E0004C0210924B0210924A021092490285E68D
:1000F00090E09093500280934F0280913F028B31A9
:1001000008F049C021E230E030934A0220934902CE
:1001100023E630E030934C0220934B0222E430E09F
:1001200030934E0220934D022091680094E0883075
:1001300038F091E0803120F092E0873108F098E0CB
:10014000922B909368002DE630E0883070F02BE61B
:1001500030E0803150F02CE630E0873130F02AE694
:1001600030E08B3110F030E020E0309347022093F4
:100170004602803108F03FC0877091E001C0990FBE
:100180008A95EAF7892F8093480280914F029091D7
:1001900050020197F1F780914D0290914E02892B08
:1001A00049F1E0913102F091320282E0E333F80745
:1001B00009F1309739F0A389B4899C91858980959C
:1001C00089238C93809151028E7F809351021092EB
:1001D000300210922F0283E392E0909332028093D8
:1001E0003102E0914602F0914702808190914802ED
:1001F000892B80830895803179F0282F30E0873172
:1002000040F42151310981E001C0880F2A95EAF7B5
:10021000BACF27513109F7CF80E8B5CFCF92DF921F
:10022000EF92FF920F931F93CF93DF936C01EB013B
:100230007B01E40EF51E10E000E0CE15DF0561F055
:100240006991D601ED91FC910190F081E02DC601FC
:100250000995080F191FF1CFC801DF91CF911F91A8
:100260000F91FF90EF90DF90CF9008953FB7F894F3
:100270008091270290912802A0912902B0912A0230
:1002800026B5A89B05C02F3F19F00196A11DB11DF1
:100290003FBFBA2FA92F982F8827BC01CD01620F2D
:1002A000711D811D911D43E0660F771F881F991FE7
:1002B0004A95D1F70895CF92DF92EF92FF92CF93B4
:1002C000DF936B017C01D2DFEB01D0DF6C1B7D0B78
:1002D000683E7340A0F0C114D104E104F10439F484
:1002E000DF91CF91FF90EF90DF90CF90089581E064
:1002F000C81AD108E108F108C851DC4FE6CFC11493
:10030000D104E104F10409F7EBCF209131023091DF
:1003100032022817390781F490912F028091300220
:10032000981751F0E0912F02F0E0EE51FE4F8081DE
:10033000082E000C990B08958FEF9FEF08952091E0
:100340003102309132022817390739F48FB7F89407
:100350001092300210922F028FBF0895EF92FF92F9
:100360000F931F93CF93DF93DC015C96ED90FC908D
:100370005D97E114F10479F481E090E013969C9389
:100380008E93129790E080E0DF91CF911F910F91B3
:10039000FF90EF9008955196ED91FC9152975096F1
:1003A0008C915097982F90950FB75E962C915E97F1
:1003B000122F127021FD6095F8942081112319F1FC
:1003C000282B2083E7012197F1F728E0462F50E002
:1003D000308160FF1AC0382B3083E7012197F1F795
:1003E000BA0175956795215089F7112381F08081B5
:1003F000892380830FBF5C968D919C910197F1F7C3
:1004000081E090E0C1CF2923DCCF3923E5CF908173
:10041000892BEFCFCF93DF936DE083E392E09EDFF4
:10042000EC016AE083E392E099DF8C0F9D1FDF917E
:10043000CF91089520913102309132022817390767
:1004400069F48091300220912F0290E0805C9F4FF0
:10045000821B910960E470E007D4089590E080E089
:100460000895209131023091320228173907B9F4EA
:1004700090912F0280913002981789F0E0912F021D
:10048000F0E0EE51FE4F808120912F0230E02F5F8F
:100490003F4F2F73332720932F0290E008958FEF63
:1004A0009FEF0895CF93DF93EC01809152029091DA
:1004B0005302009759F020915402309155022C17A5
:1004C0003D0720F081E0DF91CF910895BE016F5F7D
:1004D0007F4F3ED5009789F090935302809352024C
:1004E000D0935502C0935402209156023091570286
:1004F000232B41F7FC011082E5CF80E0E4CFFC0123
:1005000001900020E9F73197AF01481B590BBC015E
:1005100083E392E083CECF93DF93F1DFEC017ADFC8
:100520008C0F9D1FDF91CF9108958F929F92AF9274
:10053000BF92EF92FF920F931F93CF93DF93CDB7AC
:10054000DEB7A1970FB6F894DEBF0FBECDBF162F52
:10055000042F19A2423008F40AE07E0121E2E20EE3
:10056000F11C802E912CB12CA12C612FA50194019E
:100570008ED3802F622F38D3181B1A30F4F4105DFD
:10058000F70112937F01122F732FCA01232B242B03
:10059000252B59F7CF01B3DFA1960FB6F894DEBF34
:1005A0000FBECDBFDF91CF911F910F91FF90EF90C4
:1005B000BF90AF909F908F900895195CE1CF1F92EC
:1005C0000F920FB60F9211242F933F938F939F9307
:1005D000AF93BF938091230290912402A0912502B2
:1005E000B09126023091220226E0230F2D3768F1C8
:1005F00029E8230F0396A11DB11D209322028093A9
:10060000230290932402A0932502B09326028091A6
:10061000270290912802A0912902B0912A02019606
:10062000A11DB11D8093270290932802A093290257
:10063000B0932A02BF91AF919F918F913F912F91DB
:100640000F900FBE0F901F9018950296A11DB11D1F
:10065000D4CF1F920F920FB60F9211242F933F9376
:100660004F935F936F937F938F939F93AF93BF93BA
:10067000EF93FF93E0913102F0913202309749F00D
:10068000A685B7858585968D91FF14C09C91892399
:10069000A1F4FF91EF91BF91AF919F918F917F91C5
:1006A0006F915F914F913F912F910F900FBE0F90DF
:1006B0001F9018959C91892361F7A389B4899C9117
:1006C0008589809589238C93868997890197F1F78D
:1006D000608D718DA685B785558538E020E0CB010A
:1006E0000197F1F7822F90E095958795282F4C91EF
:1006F000452309F02068315091F7868D81FD2095C2
:100700008091300290E001968F73992730912F02EB
:10071000381799F0A0913002B0E0AE51BE4F2C9343
:1007200080933002828D938D0197F1F7A389B4896C
:100730008C919589892B8C93ACCF868D8160868F27
:10074000F1CF90E0FC01E659FF4F3491FC01E25BF0
:10075000FF4F2491FC01EE5CFF4FE491EE23D1F0BA
:10076000332339F03330B9F4809180008F77809350
:100770008000F0E0EE0FFF1FE85DFF4FA591B49100
:100780008FB761110EC0F8949C91E22FE095E92398
:10079000EC938FBF0895343061F7809180008F7D96
:1007A000E6CFF894EC91E22BF3CFCF93DF9300D018
:1007B000CDB7DEB793E095BD789480916E008160EF
:1007C00080936E0081E0809380009093810086E8A2
:1007D00080937A0080DC8AEF90E0A0E0B0E0809324
:1007E000370290933802A0933902B0933A0283E320
:1007F00092E0A5DD68EE73E080E090E05CDD8AE1E8
:1008000091E089DE88E591E086DE8AE191E083DE91
:1008100083E392E094DD64E670E080E090E04BDDFD
:1008200080912D0290912E02892B61F48AE791E04C
:1008300066DE80912D0290912E02019690932E02F9
:1008400080932D0280912D0290912E02029761F4E7
:1008500084E991E054DE80912D0290912E02019660
:1008600090932E0280932D0283E392E0E3DD18162D
:100870001906B4F600912D0210912E0204301105D4
:1008800078F683E392E0EDDD90932C0280932B02C7
:10089000AC01405351094A30510508F05AC08983D0
:1008A0001A8200915602109157020F5F1F4FC80124
:1008B000F9DD882391F0209152023091530280910A
:1008C000560290915702BE016F5F7F4F820F931FB8
:1008D000FED3109357020093560280912B02909101
:1008E0002C020A9709F680912D0290912E0203970F
:1008F00009F0BACF86EC91E002DE8091520290912D
:100900005302009709F47DC027D1709301016093D1
:100910000001882799274AE008DE7CDD609100010C
:1009200083E390E054D16AEF70E080E090E0C3DCB4
:100930006FEF8CE390E04BD180912D0290912E02CD
:10094000019690932E0280932D028EED91E0D7DDDB
:100950008BCF0A9711F60130110509F0BECF8EEA50
:1009600091E0CDDD80915202909153020097E1F128
:10097000F3D07093030160930201882799274AE01E
:10098000D4DD48DD6091020182E390E020D183E371
:1009900092E0D5DC60E971E080E090E08CDC9BDBEC
:1009A00090E080E07FDD209152023091530281116E
:1009B0001FC02115310511F0C90141D21092530217
:1009C0001092520210925702109256021092550243
:1009D0001092540280912D0290912E0201969093D4
:1009E0002E0280932D0279CF60E070E0CB01C1CF61
:1009F000109257021092560263E971E0C90167D361
:100A0000E9CF60E070E0CB0180CF109253021092EA
:100A100052021092550210925402109257021092F4
:100A2000560290E080E03EDD209152023091530268
:100A3000811169C02115310511F0C90100D2109250
:100A400053021092520210925702109256021092C4
:100A5000550210925402109236021092350288EE1E
:100A600093E0A0E0B0E08093370290933802A09327
:100A70003902B0933A028EE091E090933402809371
:100A8000330210924A021092490210924C021092C4
:100A90004B0210924E0210924D0210925002109290
:100AA0004F02609151026E7F6D7F60935102669597
:100AB000617081E0682786E044DE8FB7F894569A2B
:100AC0008FBF80E4809343028BE290E090934502D5
:100AD000809344028FB7F89457985F988FBF8091A6
:100AE000510281FD03C061E087E02BDE87E0809347
:100AF0003F0280E88093400289E290E090934202B6
:100B0000809341020895109257021092560263E9B1
:100B100071E0C901DCD29FCF8EE091E09093340266
:100B2000809333028091310290913202835392403C
:100B300071F4E0914602F091470290818091480261
:100B40008095892380831092320210923102809125
:100B500052029091530273C11F93FC019927882779
:100B6000BC01E89411911032E9F3193010F01E30F5
:100B7000C8F31B3249F01D3241F4689405C012D00D
:100B8000610F711D811D911D119110531A30B8F321
:100B90003EF490958095709561957F4F8F4F9F4F54
:100BA0001F910895592F482F372F262F660F771F33
:100BB000881F991F660F771F881F991F620F731F69
:100BC000841F951F660F771F881F991F0895262F72
:100BD000F999FECF1FBA81BD20BD0FB6F894FA9ADD
:100BE000F99A0FBE01960895002480FD060E660F47
:100BF00011F08695D1F7802D08952F923F924F9254
:100C00005F926F927F928F929F92AF92BF92CF929C
:100C1000DF92EF92FF920F931F93CF93DF93CDB7A5
:100C2000DEB7CA1BDB0B0FB6F894DEBF0FBECDBF1D
:100C300009942A88398848885F846E847D848C84EE
:100C40009B84AA84B984C884DF80EE80FD800C81F7
:100C50001B81AA81B981CE0FD11D0FB6F894DEBFDA
:100C60000FBECDBFED01089597FB072E16F400943B
:100C700006D077FD08D02DD007FC05D03EF4909526
:100C800081959F4F0895709561957F4F0895A1E2DA
:100C90001A2EAA1BBB1BFD010DC0AA1FBB1FEE1FF6
:100CA000FF1FA217B307E407F50720F0A21BB30B41
:100CB000E40BF50B661F771F881F991F1A9469F7BD
:100CC00060957095809590959B01AC01BD01CF0119
:100CD0000895AA1BBB1B51E107C0AA1FBB1FA61783
:100CE000B70710F0A61BB70B881F991F5A95A9F7D5
:100CF00080959095BC01CD010895EE0FFF1F0590E2
:100D0000F491E02D09940F931F93CF93DF938230DA
:100D1000910510F482E090E0E0915A02F0915B02BC
:100D200030E020E0B0E0A0E0309799F421153105E3
:100D300009F44AC0281B390B24303105D8F58A81C3
:100D40009B816115710589F1FB0193838283FE010B
:100D500011C0408151810281138148175907E0F089
:100D60004817590799F4109761F012960C9312974F
:100D700013961C933296CF01DF91CF911F910F9163
:100D8000089500935A0210935B02F4CF21153105A8
:100D900051F04217530738F0A901DB019A01BD0158
:100DA000DF01F801C1CFEF01F9CF90935B0280938F
:100DB0005A02CDCFFE01E20FF31F8193919322508F
:100DC000310939832883D7CF2091580230915902B5
:100DD000232B41F4209106013091070130935902F1
:100DE000209358022091040130910501211531050D
:100DF00041F42DB73EB74091080150910901241BE1
:100E0000350BE0915802F0915902E217F307A0F474
:100E10002E1B3F0B2817390778F0AC014E5F5F4F50
:100E20002417350748F04E0F5F1F50935902409327
:100E30005802819391939FCFF0E0E0E09CCFCF9355
:100E4000DF930097E9F0FC01329713821282A091A0
:100E50005A02B0915B02ED0130E020E01097A1F45E
:100E600020813181820F931F2091580230915902C5
:100E70002817390709F061C0F0935902E09358022E
:100E8000DF91CF910895EA01CE17DF07E8F54A8197
:100E90005B819E0141155105B1F7E901FB83EA83AE
:100EA00049915991C40FD51FEC17FD0761F480815A
:100EB00091810296840F951FE9019983888382812D
:100EC00093819B838A83F0E0E0E012968D919C9160
:100ED00013970097B9F52D913C911197CD0102968A
:100EE000820F931F20915802309159022817390719
:100EF00039F6309751F510925B0210925A02B09376
:100F00005902A0935802BCCFD383C2834081518140
:100F1000840F951FC817D90761F44E5F5F4F888112
:100F20009981480F591F518340838A819B81938304
:100F300082832115310509F0B0CFF0935B02E09375
:100F40005A029ECFFD01DC01C0CF13821282D7CF9F
:100F5000B0E0A0E0EDEAF7E052CE8C01009741F45A
:100F6000CB01D1DE8C01C801CDB7DEB7E0E163CEA5
:100F7000FC01E60FF71F9C0122503109E217F3072D
:100F800008F499C0D901CD91DC911197C617D70704
:100F900090F0C530D10538F3CE0104978617970736
:100FA00010F3C61BD70B2297C193D1936D937C93FB
:100FB000CF0145DFD8CF5B01AC1ABD0A4C018C0EC6
:100FC0009D1EA0915A02B0915B02512C412CF12C34
:100FD000E12C109731F580915802909159028815B3
:100FE000990509F05CC04616570608F058C0809174
:100FF000040190910501009741F48DB79EB740918F
:10100000080150910901841B950BE817F90708F0B6
:1010100052C0F0935902E0935802F9017183608342
:10102000A2CF8D919C91119712966C901297139666
:101030007C901397A815B90559F56C0142E0C40ED0
:10104000D11CCA14DB0420F1AC014A195B09DA0196
:101050001296159780F06282738251834083D90182
:101060006D937C93E114F10471F0D7011396FC9316
:10107000EE93129778CF22968C0F9D1FF9019183E2
:101080008083F301EFCFF0935B02E0935A026BCFC2
:101090004816590608F42C017D01D3019ACFCB01E3
:1010A00032DE7C01009739F0AE01B80107D0C801EB
:1010B000C6DE870158CF10E000E055CFFB01DC0110
:1010C00002C001900D9241505040D8F70895FB01A5
:1010D000DC0101900D920020E1F7089510E0C4E4D6
:1010E000D0E003C0FE0109DE2196C534D107D1F757
:0410F000F894FFCFA2
:1010F400FF00FF0000005C02800000000000AE0161
:101104000E011A02310285019F013D3D3D3D3D3DE9
:101114003D3D3D3D3D3D3D3D3D3D3D3D3D3D3D3DFB
:101124003D3D3D3D3D3D3D3D3D3D3D3D3D3D3D3DEB
:101134003D3D3D3D3D3D3D3D3D3D3D3D3D3D3D3DDB
:101144003D3D3D3D3D3D3D004D6963726F636F6EB6
:1011540074726F6C6C657220415454696E7920739B
:101164007461727465642E2E2E00496E73657274F8
:101174002076616C75652072656769737465722089
:1011840035300A00496E736572742076616C75653A
:101194002072656769737465722035310A0057726D
:1011A4006974696E67207265676973746572203546
:1011B4003020746F200057726974696E67207265FD
:1011C40067697374657220353120746F20004F4B4A
:0211D4000A000F
:00000001FF
